:1000000040C05AC059C058C057C056C055C054C04F
:1000100053C053C051C050C04FC04EC04DC04CC063
:100020004BC04AC049C048C047C046C045C044C094
:1000300043C042C0C0F9A4B0999282F880908883EE
:10004000C6A1868EC289CFE18FC7C8ABA38C98AFFB
:100050009287C1E3818991A4FF00020207FF080C87
:1000600017F0F1EF0001100001100F11000E121F28
:10007000210007FF0B060803060603050704050316
:10008000060011241FBECFEFD4E0DEBFCDBF11E0CC
:10009000A0E0B1E0EEE7F3E102C005900D92A430DC
:1000A000B107D9F714E0A4E0B1E001C01D92A83374
:1000B000B107E1F720D761C9A3CF1F920F920FB606
:1000C0000F9211242F933F934F935F936F938F93CE
:1000D0009F93AF93BF93EF93FF9313BE90918D01C6
:1000E000937083B18770873061F09F5F90930601B2
:1000F0009150199904C09B5F9093060195501A9BEB
:1001000061C0933009F466C080918D0190918E0199
:10011000A0918F01B09190010196A11DB11D809316
:100120008D0190938E01A0938F01B0939001682F61
:10013000E82FE37088B18F6088B9EE2399F12091A0
:100140000701220F2093070187B1807F822B87B997
:100150008091FB03382F80FF02C067FD4FC04E2FF8
:1001600050E0FA01E450FC4F80818BB932FD1FC092
:1001700031FF02C066FD5F9888B120952F70807FA7
:10018000282B28B9FF91EF91BF91AF919F918F914B
:100190006F915F914F913F912F910F900FBE0F90F4
:1001A0001F90189581E08093070121E0CDCF8091C9
:1001B0008E0190E08370907048175907E1F231FD8D
:1001C000D9CFDACF20910601285F20930601933022
:1001D00009F09ACF8091040187FD1AC02091060191
:1001E000222379F480910501882319F08AEF809306
:1001F0000401209305011092060186CF8FEF8BB981
:10020000BBCF90910501992349F420930901F1CFC7
:100210008F5F8093040120910601EBCF291749F7E6
:100220008F5F80930401853124F32093090110929C
:100230000401DFCF982F862F81568A31B0F0862FA8
:1002400081548A3130F060536A3098F4E62FF0E040
:1002500003C06753E62FF0E0EC5CFF4F8491E92F79
:10026000F0E0E450FC4F808308956755E62FF0E0FE
:10027000F3CFE4E2F0E0F0CF80910901882339F474
:1002800097E093BF8895809109018823D1F38091ED
:10029000090110920901805D0895F894E1E6F0E00B
:1002A00080E88083108210927A0083E88093640053
:1002B00014B887E085B917B88FE088B98FEF8BB98C
:1002C0008AB9E1EBF0E0808185608083E0E7F0E0CF
:1002D0008081816080837894089560E280E0AADF65
:1002E00060E281E0A7DF60E282E0A4DF60E283E019
:1002F000A1DF08958091FC038F778093FC038091A8
:10030000FD038F778093FD038091FE038F778093A9
:10031000FE038091FF038F778093FF0308958093FE
:10032000FB0308952F923F924F925F926F927F92BC
:100330008F929F92AF92BF92CF92DF92EF92FF92F5
:100340000F931F93DF93CF93CDB7DEB72E970FB6E2
:10035000F894DEBF0FBECDBF85EFC82E83E0D82E48
:1003600000E8702E11E0412E512CB7E82B2EB2E0A0
:100370003B2EA0E4AA2EAFE1BA2E209101013091CC
:100380000201C90182979093020180930101815972
:10039000914048F5309302012093010180910C04B3
:1003A00090910D04909581959F4F90933204809386
:1003B0003104C216D30609F4D2C080912B048823DD
:1003C00009F0CAC0AAE0B4E0F90182E201900D92FE
:1003D0008150E1F780913104909132049093170499
:1003E00080931604E4C020918B0130918C018091A0
:1003F00036049091370490930D0480930C048091FF
:100400002E0490912F0490930F0480930E048091FA
:100410002C048093180480913504809319048091F2
:10042000FA0380931A048091020480932B042150D4
:10043000304030930B0420930A044091F90358E1B3
:1004400045274093F90310922A041092290420E0D2
:1004500080911A04422F4F5F40931E04281708F022
:1004600045C08091290480931D04809323048091CA
:100470002A04807880931F04433008F494C080914C
:100480000101909102019C01D901EAE0F4E082E2CD
:1004900001900D928150E1F720910C0430910D04F0
:1004A00088279927821B930B90938C0180938B0153
:1004B000C201821B930B9093370480933604809182
:1004C0000E0490910F04909581959F4F90932F0467
:1004D00080932E0470922C041092350480911E0497
:1004E00083508093FA031092020447CF433008F4FC
:1004F0004FC020E030E08091F5039091F6038054E6
:100500009F4109F432C28091190490E028233923D5
:10051000232B09F4FCC180918D0190918E01A09153
:100520008F01B0919001B7FDE7C32091290420937A
:10053000F5031092F60390912A04892F8777809310
:100540002D0483E080931E0420931D042093230434
:10055000907890931F0493CF813009F4D7C02E96E2
:100560000FB6F894DEBF0FBECDBFCF91DF911F91C4
:100570000F91FF90EF90DF90CF90BF90AF909F9042
:100580008F907F906F905F904F903F902F90089545
:100590008091290480931D048093230480912A0470
:1005A000807880931F04B0921704A0921604809163
:1005B00016049091170422273327281B390B8091AA
:1005C0000C0490910D042817390724F08091300411
:1005D000843238F080911E04833008F4C1C120ECCD
:1005E00030EE30931104209310044091F903609190
:1005F0002304E62FF0E0E65FFE4F208120932104E4
:10060000822F842321F1722F7770709322047093CC
:100610001B04E72FF0E0EF58FF4FE491E0931C0438
:1006200080911B04733010F087FD6DC1E0911C04B4
:10063000EF5FE0931C04F0E0EF59FF4FE491E19588
:10064000E0931B04EE2309F03EC160912304862F42
:10065000875F87778093230490911D04891709F0A1
:10066000C6CF2091100430911104C9018854914ED5
:1006700081579D4318F052E650931E0440E050E02D
:10068000809116049091170480549F4109F47DC114
:10069000205C304E422B532B20543F41452B09F414
:1006A0006DC1309311042093100420911E04809199
:1006B000080190911904892390E040E050E0233034
:1006C00008F059C184239523892B09F4C1CE609188
:1006D000290467706F5980E0ADDD8091290482950F
:1006E0008F7068E3681B81E0A5DD60912A04677064
:1006F0006F5982E09FDD80912A048295877068E3BC
:10070000681B83E097DD20911E04A2CEAAE0B4E02E
:10071000F90182E201900D928150E1F7809131045C
:1007200090913204909581959F4F909334048093DB
:100730003304209133043091340440E080910A0462
:1007400090910B04821793070CF441E090912004E0
:100750009F5F90932004442309F451C080911E04AC
:10076000981708F04CC02091120430911304809126
:100770002004833040F48091140490911504821772
:1007800093070CF085C380910101909102019C01B7
:10079000D901EAE0F4E082E201900D928150E1F7A4
:1007A00080910C0490910D04909581959F4F9093AA
:1007B0008C0180938B018091140490911504909585
:1007C00081959F4F90933704809336048091120453
:1007D00090911304909581959F4F90932F0480934F
:1007E0002E048091250480932C041092350480916E
:1007F00020048093FA0381E080930204BECD3093FD
:1008000013042093120480911904882309F4C0C0B2
:100810004091F5035091F6039FE14034590709F4E4
:10082000B7C0205C304E09F4B3C080912304282F58
:1008300030E04217530709F467C2E0912604F0E064
:10084000E65FFE4F4091F9034A5F40834650A09116
:100850002504B0E0E0912404F0E0E65FFE4F108252
:10086000A65FBE4F1C92265F3E4F80912104F90186
:100870008083E0912704F0E0E65FFE4F809128043A
:10088000808360912304209112043091130480919D
:100890001004909111048217930774F4309311049B
:1008A000209310046093290480912504807890910E
:1008B0002404892B80932A0480911F04882309F43F
:1008C0006CC010921F0460932404709226047092EE
:1008D000250480911F048F83882309F052C0509112
:1008E0001B0480912404580F509324045093270430
:1008F000052F10E0852F887809F4B0C0709122048C
:10090000609123048DCE819580931B04DCCF4091B0
:10091000F903B8E14B274093F9032091010130918D
:1009200002012E5D3F4F309302012093010140915F
:1009300010045091110460E070E080910E049091D9
:100940000F0448175907A4F0CB01840F951F90930B
:10095000110480931004909332048093310429CDC4
:1009600020910E0430910F043CCE21E030E0CBCD3D
:1009700061E070E0E9CF41E050E0A4CE20E030E05B
:1009800090CE50912A045827AFCF41E050E080CE5E
:1009900080912304282F30E050CF10911B04F09059
:1009A0002404009121047091220480911C0490E0A1
:1009B0000797272F30E024503040822B932B892B30
:1009C00091F46D5F212F2595277026276350209382
:1009D0002604E22FF0E0E65FFE4F808190E0841B6A
:1009E0009109069751F151E0212F332727FD3095CA
:1009F0002F193109260F311D802F90E080729070E1
:100A0000282B392B80E0733008F081E05823852FA4
:100A100090E0282B392B232B09F46BC190E0753023
:100A200008F491E080912804980F90932804809115
:100A30002804882309F44DCFF3CDA2E0A227B0E02B
:100A4000A65FBE4FF1E02F27E22FF0E0E65FFE4FFA
:100A50008C919081892B39F650E0C6CFA091180473
:100A60002A2F30E0F901E65FFE4F808190E02058A8
:100A700030408223932320583F4F892B31F0C80107
:100A8000821B930B02970CF47CC180901004909011
:100A900011049092110480921004709122041E821D
:100AA000733040F491E09E835A1721F4A0E15A2755
:100AB0005093270480912704E82FF0E0E65FFE4F73
:100AC000FC87EB87608060922804E62EFF24A0E07C
:100AD000B0E0662011F4A1E0B0E020E030E0C80111
:100AE0008E199F0987709070892B11F421E030E0F6
:100AF0002A1B3B0B80E090E0733010F481E090E023
:100B000028233923862D842390E0282B392B232B6F
:100B100009F086CD262D30E0F901E770F070E75A34
:100B2000FF4F85919491F5E28F02F0011124207C12
:100B30003070E20FF31FFE87ED87F0930104E0931E
:100B40000004F7FD19C190921104809210042091C5
:100B50001E042B8380910C0490910D048816990635
:100B60001CF0223008F07DCD3B81313009F495C175
:100B700080910E0490910F049093130480931204BB
:100B80005B81852F90E08A1B9B0B02970CF47BCE38
:100B9000763008F404C1A0E0B0E09701265F3E4F34
:100BA000C801865F9E4F9A878987B0931304A093EC
:100BB00012048091260490E0F9011082EB85FC85F7
:100BC0001082FC01E65FFE4F108250912104252F18
:100BD0002062E985FA852083887869F4E09125040C
:100BE000F0E0E65FFE4F4A5F40834650D296B093F6
:100BF0001304A0931204E0911204F0911304272F20
:100C000030E03A83298330913004388789819A8192
:100C1000049720E030E0A885AE3110F021E030E00C
:100C2000822B932B892B09F0B7C084E190E09F01C0
:100C3000281B390B3093130420931204BE81BB236D
:100C400009F0BEC0409100045091010480910E044F
:100C500090910F042091120430911304820F931F7E
:100C6000840F951F909313048093120420910A041B
:100C700030910B04C401821693060CF4C9019093C1
:100C800015048093140490E0BB81B63008F091E025
:100C900080E0733008F081E0982380E0662009F45A
:100CA00081E0892390E0EF81EE2309F491E089232C
:100CB000FB81F1504F2F481BFF5FFB8320E03885FD
:100CC0003E3108F021E080E05B81533008F481E0A0
:100CD000282B30E0809116049091170480549F4196
:100CE000282B392B232B09F04B836B816093200435
:100CF0003ACDF09225049BCE423608F016CC2091D6
:100D0000290490912A0420CC9091240480912D04F0
:100D1000981709F092CD80910E0490910F04909550
:100D200081959F4F2091000430910104821B930B09
:100D30009093F8038093F70380912504809308042F
:100D4000220F232F221F330B80913004820F8093B8
:100D5000300420910101309102012E5D3F4F30930C
:100D600002012093010180910C0490910D04909355
:100D70003204809331041DCBE0E48E2EEFE19E2EF1
:100D8000E2CE201B310B223031050CF07ECEF0E498
:100D90008F2EFFE19F2E7DCE80E090E048CF97011F
:100DA000265F3E4FD90118968C91A82FB0E0F8012C
:100DB000E65FFE4FFA87E9878085A81BB109F5CE6B
:100DC000F70132978E2F887809F484C0E1E0F0E0D3
:100DD000FD83EC83F70132968E2F887809F46DC07D
:100DE000A1E0B0E0BC87AB87888586958695D90160
:100DF000A80FB11DEE24FF24F0E16F27E62FF0E0ED
:100E0000E65FFE4F208130E0842F90E08496281723
:100E1000390709F46CC092012E193F098C819D811C
:100E2000281B390BEB85FC852E1B3F0BC901880F56
:100E3000991F880F991F880F991F820F931FA80F62
:100E4000B91FB0931304A093120480911B04992737
:100E500087FD9095800F911F019687FF23C0910118
:100E600049815A81241B350B3093150420931404B7
:100E7000A985BA858C91820F8C9340910004509182
:100E80000104420F531F5093010440930004DECE2F
:100E900030933404209333044CCC8D859E85871B7E
:100EA00091096ACE252F30E020723070005F1F4F0D
:100EB00020233123220F331FD7CF1C861B86E65FEA
:100EC000FE4F8081581709F48FCFE1E0F0E0FC87F6
:100ED000EB878ACF1D821C82E65FFE4F8081581708
:100EE00009F478CF81E090E09D838C8373CF61E03B
:100EF000E62EF12C90CF7F928F929F92AF92BF926D
:100F0000CF92DF92EF92FF920F931F93CF93DF93D5
:100F1000C4D917E002E1B9E0FB2EC0E8DFEFA8E397
:100F2000EA2EF4E0DF2EE5E0CE2E70ECA72E70EE78
:100F3000B72E60E4862E6FE1962E5BE3752E10923D
:100F4000FB0363E580E076D968E481E073D961E46E
:100F500082E070D968E483E06DD980E18093F90381
:100F6000109230041092F8031092F70310920804C4
:100F7000EAE0F1E0119281E0EB38F807D9F727E0D9
:100F800076E002C0272F782F30E0C90187589F4FA5
:100F9000FC018491885FF901E65FFE4FE059FF4F45
:100FA0008083E057F040885F8083008BE05AFF4FDA
:100FB000F082D901189624503040229F202D112410
:100FC00087E066E090E0880F991FFC01EE0FFF1F9D
:100FD000EE0FFF1FEE0FFF1FEA0FFB1FE65FFE4F36
:100FE0000797889FA001899F500D989F500D11244D
:100FF00057FDBDC15595479555954795822F840F4F
:101000008083862F61506E3FE9F6872F81508E3F97
:1010100009F0B8CF8FEF80932D04D092090494E0AB
:10102000292F30E080910901882331F413BF88957E
:10103000809109018823D1F380910901805D10928C
:101040000901F901ED5FFB4F8083893309F4A2C0E8
:10105000893398F420FD02C0805D8083943009F4C8
:1010600009C1953009F4BCC06081892FE3D8909103
:1010700009049F5F90930904D3CF8A3309F4AEC06B
:101080008B3341F7209103042B3309F439C130E04D
:10109000215E3C4F8091040490E082959295907F70
:1010A0009827807F9827281B390B3093F6032093CD
:1010B000F50320910504215E8091060490E082955D
:1010C0009295907F9827807F9827281B20932D0446
:1010D000B0928C01A0928B019092370480923604DA
:1010E0008091F7039091F80390932F0480932E043E
:1010F0008091080480932C0481E08093350483E080
:101100008093FA03109202040DD91092FB03809190
:1011100003048B3309F4CBC02091310430913204A5
:10112000FFE120343F0709F0B1C08091FC038F77C5
:101130008093FC038091FD038F778093FD03809162
:10114000FE038F778093FE038091FF038F77809358
:10115000FF0370920304225C304E0CF05ECF6DE40E
:1011600080E068D861E481E065D864E582E062D817
:1011700064E583E05FD880910901882331F413BFCF
:101180008895809109018823D1F3809109011092FB
:101190000901D5CE66E480E04DD86EE481E04AD8FE
:1011A00060E282E047D860E283E044D880910901A0
:1011B000882331F413BF8895809109018823D1F3E6
:1011C00080910901805D1092090180932D04823382
:1011D000C9F08333C9F1813309F4B1CEC092090457
:1011E0007CD81092090490E01BCF90910901892FBF
:1011F000805D1092090180932D048B3379F3915017
:101200009093000163E580E015D864E581E012D891
:10121000609100016F5C83E00DD880910901882303
:1012200021F713BF8895809109018823D1F3DDCF81
:1012300080910901805D1092090180932D048B3308
:1012400069F281708093080168E480E0F3D766E575
:1012500081E0F0D760910801605D83E0EBD7809179
:101260000901882329F713BF8895809109018823F4
:10127000D1F3DECF32D8609107046093030480E09D
:10128000D9D781E08093090491E0CACE6AE580E075
:10129000D1D765E581E0CED767E482E0CBD760E2C5
:1012A00083E0C8D7209131043091320452CF60914D
:1012B000F50367706F5980E0BDD78091F503909179
:1012C000F603959587959595879595958795959529
:1012D00087956E2D681B81E0ADD760912D046770F6
:1012E0006F5982E0A7D780912D04829587706E2D6B
:1012F000681B83E09FD720913104309132042BCFBB
:101300009092F6038092F503F894CE0100900001CC
:1013100002C0880F991F0A94E2F7AA2797FDA095AB
:10132000BA2F80938D0190938E01A0938F01B0937B
:1013300090017894D2D7809108018823D9F08091C8
:10134000FC038F778093FC038091FD038F7780935C
:10135000FD038091FE038F778093FE038091FF034E
:101360008F778093FF0381E08093FB03B1CE4D5FC5
:0E1370005F4F40CED092FB03ABCEF894FFCF80
:04137E0002F5030071
:00000001FF
